:0A0000008316FF23900083012C2BD0
:100658008301862B8312A1002108A000013003101A
:10066800A00DFF3E031D332B0310200D01389F0002
:100678000930A000A00B3E2B412B83129F14442B62
:100688009F18472B482B442B492B08008312A100A5
:100698001F30A000200885053F30A000A00B522B7A
:1006A800552B8312A20108302202031C5C2B5D2B00
:1006B8005F2B7F2B7F2B211C622B632B652B8516D1
:1006C8006C2BDF30A000200885056A2B6B2B6C2B68
:1006D80003108312A10C3C30A000A00B712B640006
:1006E80001308312A0002008A20708302202031C50
:1006F8007E2B7F2B5F2B85164030A000A00B822B12
:10070800640008008312A501A9010730831685003B
:1007180083129F01573083169F0064002030831294
:100728008500962B8312A501AA30A3002308A900EF
:10073800AA0103302A02031CA22BA32BA52BD22B20
:10074800D22B2A082E23803083121E020318AD2BC9
:10075800AE2BB82B1E087F3AA3002A08263E840039
:10076800230883138000C02B1E08A3002A08263EF6
:1007780084002308831380002A08263E840000088A
:10078800A3002308A9070130A3002308AA07033000
:100798002A02031CD02BD12BA52BD22BAA304A23FB
:1007A8008312AA0103302A02031CDB2BDC2BDE2B6D
:1007B800F02BF02B2A08263E8400831300084A23D6
:1007C80001308312A3002308AA0703302A02031C5E
:1007D800EE2BEF2BDE2BF02B29084A231630831241
:1007E800A400D030A300A30BF72BA40BF72B6400B5
:0607F800962B962B002851
:02400E008431FB
:00000001FF
